:100000000C94E4020C9419150C94F2140C940C0347
:100010000C940C030C940C030C94870B0C940C03A1
:100020000C940C030C940C030C940C030C940C0314
:100030000C940C030C940C030C940C030C940C0304
:100040000C94A8140C940C030C9466150C94401595
:100050000C940C030C940C030C940C030C940C03E4
:100060000C940C030C940C0354534D3A494E4954D0
:100070000A002154534D3A494E49543A54535020A2
:100080004641494C0A0054534D3A494E49543A545A
:100090005350204F4B0A0054534D3A465041520A98
:1000A000002154534D3A465041523A4E4F2052454A
:1000B000504C590A002154534D3A465041523A4649
:1000C00041494C0A0054534D3A465041523A4F4B25
:1000D0000A0054534D3A49443A5245510A00545388
:1000E0004D3A49440A002154534D3A49443A464155
:1000F000494C0A0054534D3A49443A4F4B0A005474
:10010000534D3A55504C0A002154534D3A55504CDA
:100110003A4641494C0A0054534D3A55504C3A44E2
:100120004757432C4F3D25642C4E3D25640A00540F
:10013000534D3A55504C3A4F4B0A0054534D3A5296
:10014000454144593A49443D25642C5041523D258E
:10015000642C4449533D25640A002154534D3A52BE
:10016000454144593A55504C204641494C2C534E38
:10017000500A0054534D3A4641494C3A5044540AAF
:100180000054534D3A4641494C3A434E543D256440
:100190000A0054534D3A4641494C3A52452D494E76
:1001A00049540A004D434F3A50494D3A4E4F444549
:1001B000205245473D25640A00215453463A4D5389
:1001C000473A52454C204D53472C4E5245500A0059
:1001D0005453463A4D53473A42430A005453463A21
:1001E0004D53473A41434B0A00215453463A4D532D
:1001F000473A504F4E4720524543562C494E4143B3
:10020000544956450A005453463A4D53473A504FC5
:100210004E4720524543562C48503D25640A005411
:1002200053463A4D53473A50494E4745442C49446A
:100230003D25642C48503D25640A00215453463A1C
:100240004D53473A4650415220494E414354495636
:10025000450A005453463A4D53473A4650415220BE
:100260004F4B2C49443D25642C443D25640A0054E1
:1002700053463A4D53473A41434B205245510A00A9
:10028000215453463A4D53473A505645522C256413
:100290003D25640A00215453463A4D53473A4C4594
:1002A0004E2C2564213D25640A005453463A4D5393
:1002B000473A524541442C25642D25642D25642C54
:1002C000733D25642C633D25642C743D25642C709E
:1002D000743D25642C6C3D25642C73673D25643A80
:1002E00025730A005453463A5349443A4F4B2C491C
:1002F000443D25640A00215453463A5349443A4642
:1003000041494C2C49443D25640A00257354534609
:100310003A4D53473A53454E442C25642D25642DC0
:1003200025642D25642C733D25642C633D25642CA8
:10033000743D25642C70743D25642C6C3D25642C23
:1003400073673D25642C66743D25642C73743D25CC
:10035000733A25730A00215453463A5254453A469B
:10036000504152204143544956450A0000000000C4
:10037000240027002A0000000000250028002B0090
:1003800000000000230026002900040404040404E3
:100390000404020202020202030303030303010234
:1003A0000408102040800102040810200102040803
:1003B00010200000000800020100000304070000F4
:1003C0000000000000004D434F3A534C503A57553F
:1003D000503D25640A004D434F3A534C503A545017
:1003E000440A004D434F3A534C503A4D533D256C0F
:1003F000750A00214D434F3A534C503A544E520A1D
:10040000004D434F3A534C503A4D533D256C752C9B
:10041000534D533D25642C49313D25642C4D313DD0
:1004200025642C49323D25642C4D323D25640A005B
:10043000214D434F3A534E443A4E4F4445204E4F80
:1004400054205245470A00215453463A534E443AE9
:10045000544E520A004D434F3A5245473A52455185
:100460000A005453463A5755523A4D533D256C7540
:100470000A004D434F3A42474E3A494E4954204FA5
:100480004B2C5453503D25640A004D434F3A42478C
:100490004E3A5354500A004D434F3A42474E3A4267
:1004A00046520A004D434F3A42474E3A494E49544C
:1004B000204E4F44452C43503D524E4E4E412D2D23
:1004C0002C5645523D322E312E300A0000407A1013
:1004D000F35A00A0724E18090010A5D4E80000E8F5
:1004E0007648170000E40B54020000CA9A3B000053
:1004F00000E1F505000080969800000040420F00E2
:100500000000A08601000000102700000000E803A2
:10051000000000006400000000000A00000000006D
:100520000100000000002C76D888DC674F0823DF2C
:10053000C1DFAE59E1B1B796E5E3E453C63AE651FF
:10054000997696E8E6C28426EB898C9B62ED407C26
:100550006FFCEFBC9C9F40F2BAA56FA5F490055AC2
:100560002AF75C936B6CF9676DC11BFCE0E40D47E7
:10057000FEF520E6B500D0ED902E0300943577050A
:100580000080841E080000204E0A000000C80C33C2
:100590003333330F986E12831141EF8D2114893B51
:1005A000E65516CFFEE6DB18D1844B381BF77C1DD1
:1005B000901DA4BBE424203284725E228100C9F124
:1005C00024ECA1E53D27BA1611241FBECFEFD8E0D9
:1005D000DEBFCDBF11E0A0E0B1E0E6E2F2E402C090
:1005E00005900D92A03FB107D9F723E0A0EFB1E04D
:1005F00001C01D92A338B207E1F712E0C4EED2E0C9
:1006000004C02197FE010E945A18C33ED107C9F7C2
:100610000E9402170C9411210C9400000F931F9359
:100620000E945F14009104021091050220910602BD
:1006300030910702601B710B820B930B1F910F917E
:1006400008959C0180910202909103028217930702
:1006500051F090910C029F7190930C023093030221
:100660002093020205C080910C02805E80930C02F0
:10067000E0910202F09103020190F081E02D3097A9
:1006800009F009950E945F146093040270930502BB
:1006900080930602909307020895EF92FF920F93C2
:1006A0001F93CF93DF93CDB7DEB7C857D1090FB6ED
:1006B000F894DEBF0FBECDBF8E010F571F4FF8015C
:1006C000E190F1908F010E945F144AE00E948B0C30
:1006D00088EA91E00E94790C9801A70168E770E030
:1006E000CE0101960E94641ACE0101960E94790CF7
:1006F00087E492E00E948012C858DF4F0FB6F8944A
:10070000DEBF0FBECDBFDF91CF911F910F91FF9044
:10071000EF900895AF92BF92CF92DF92EF92FF9247
:100720000F931F93CF93DF93EC018A8190910C027A
:1007300090FF0CC08F3F79F086E593E09F938F93F5
:100740000E944D030F900F9010E0D0C08F3F19F022
:100750000091450201C00FEF8091440288834B81D4
:1007600042FD06C046954695469517E0140F01C018
:1007700010E280E090E0892B21F080E090E00E9480
:100780000000299880E091E00197F1F76EE080E2A7
:100790000E940A1684EC90E00197F1F7602F8AE23C
:1007A0000E940A16602F80E30E940A1681EE0E94C2
:1007B0002D160F3F11F080EA01C080EB412F11325E
:1007C00008F040E220E0BE010E94D915299AE12CF0
:1007D000F12C8FEF0E942D16182F807321F481E0E9
:1007E000E81AF108B1F7299860E387E20E940A1637
:1007F00014FF03C081EE0E942D160E94201615FBE7
:10080000112710F981E00F3F09F080E0182BCE018D
:100810000E94C90B111103C0E0E4F1E002C0EDE356
:10082000F1E060910D026F702B8122FBAA24A0F8E9
:10083000322F3695369536952C81B22EB294B694D9
:1008400047E0B422CD802770DE80EA80A02FB0E0A0
:10085000F8807981111103C04FE751E002C04DE4E7
:1008600051E09F938F93FF93EF931F926F931F928B
:10087000AF921F923F931F92BF921F92CF921F92EF
:100880002F931F92DF921F92EF92BF93AF931F920D
:10089000FF921F927F935F934F938BE093E09F9320
:1008A0008F930E944D038DB79EB74E960FB6F89466
:1008B0009EBF0FBE8DBF80914502081317C0111156
:1008C00010C080E090E0892B21F085E690E00E9446
:1008D000000080910D0291E0980F9F70807F892B1E
:1008E00003C080910D02807F80930D02812FDF91E4
:1008F000CF911F910F91FF90EF90DF90CF90BF901D
:10090000AF900895CF93C82F8FEF8C0F8E3F08F5CF
:10091000C0934402C093220163E082E20E940A165F
:1009200061E081E20E940A160E9420166C2F80E08E
:1009300090E00E94C8201F92CF9384EE92E09F9394
:100940008F930E944D030F900F900F900F9081E0B6
:1009500018C01F92CF9386EF92E09F938F930E94CF
:100960004D030F900F900F900F9080E090E0892B37
:1009700021F08EE690E00E9400008FEF8093440209
:1009800080E0CF9108952F923F924F925F926F92A5
:100990007F928F929F92AF92BF92CF92DF92EF920F
:1009A000FF920F931F93CF93DF93CDB7DEB72C97B2
:1009B0000FB6F894DEBF0FBECDBFE0910202F091FA
:1009C00003020280F381E02D309709F009958091B0
:1009D0000C0284FB222720F9298784FF59C386E073
:1009E000D82E90E0E92E90E0F92E9E012F5F3F4F28
:1009F0003C832B8320EA822E26E8922EAA24A394FD
:100A0000B12C34EB432E3BE2532E31E1632E712C9B
:100A100021E041E060E070E087E10E94D91580FDAF
:100A200037C3DA94DD2009F433C3E114F10421F073
:100A300081E090E00E94000021E041E060E070E091
:100A400080E60E94D915C82E30E2381720F482EED5
:100A50000E942D16C12C21E04C2D67E473E081E645
:100A60000E94D91560E487E20E940A1680914A0329
:100A7000282F2695269526952A3108F029E182FD12
:100A800003C077E0720F01C070E280914B03877062
:100A90008D8310914C0300914803209047033090C0
:100AA000490387E493E02A877C870E94C90B2A8543
:100AB000422F50E09F938F9380914A0382FB8827B7
:100AC00080F91F928F931F922F9380914B038295F1
:100AD000869587701F928F931F921F931F922D816F
:100AE0002F9380914D031F928F931F923F921F92DD
:100AF0002F921F920F93AAEAB2E0BF93AF934A8757
:100B00005B870E944D030FB6F894DEBF0FBECDBFCA
:100B10007C854A855B85C71679F0E114F10429F0DC
:100B20008CE690E00E9400007C851F927F931F92CC
:100B3000CF9285E992E017C020914A03822F8370FB
:100B40008230E1F0E114F10421F08DE690E00E94A2
:100B500000001F9282E08F9380914A0383701F925E
:100B60008F9380E892E09F938F930E944D030F90A4
:100B70000F900F900F900F900F904ACF80910D0221
:100B8000806880930D0280914402381259C0822FF0
:100B90008695869586958A3108F089E138E0839FAD
:100BA000C00111242770822B80934A03FA01E95B6C
:100BB000FC4F178280914B0383FF21C08FE692E0A8
:100BC0009F938F930E944D0381E2E7E4F3E0A6E256
:100BD000B3E001900D928A95E1F780912A03877F17
:100BE000806180932A0380914402809327030093BD
:100BF000280386E293E00E9433160F900F909091A5
:100C00004B0394FD0BC02D81233081F480914C0364
:100C100021EF280F233008F055C0FACEACEDB1E03B
:100C2000BF93AF930E944D030F900F9020E030E0F0
:100C3000232B09F4EDCE87E493E00E940000E8CE78
:100C40003FEF331236C0A0EDB1E0BF93AF930E94E7
:100C50004D030F900F902D81233031F580910C02C0
:100C600082FF03C0173009F4D3CE183009F4D0CE78
:100C7000143109F0CDCE809145022812C9CE0E94D0
:100C80005F147370882799270E942F1010914502D6
:100C900025E143E06FEF802F0E94BA0B612F0E9485
:100CA00098150E948A03B4CE809145022812B0CED6
:100CB000BDCFA9EBB1E0BF93AF930E944D030F905E
:100CC0000F90A6CE143029F40E94660C0E94820474
:100CD0009FCE183011F510910C0210FF1BC00E941E
:100CE000660C8F3F09F494CE8F5F8F3F09F490CE4E
:100CF00090914602891708F08BCE11FD89CE809322
:100D00004602009345021F928F931F920F9383E533
:100D100092E029CF8BE392E030C01831C1F40E94F9
:100D2000660C1F928F931F920F938FE192E09F9317
:100D30008F930E944D0329E143E06FEF802F0E94C3
:100D4000BA0B61E00E9498150E948A0310CF1931F6
:100D5000B9F480910C0283FF0EC0877F80930C0250
:100D60000E94660C80930E021F928F9386E092E0A1
:100D70009F938F933CC089EE91E09F938F939DCF7B
:100D800020914803211180C18D3099F480E090E0DA
:100D9000892B21F08BE090E00E94000098E088E130
:100DA0000FB6F894A895809360000FBE90936000F2
:100DB000FFCF8B3119F50E94660C91E0811101C0C3
:100DC00090E08091100290FB80F980931002E11472
:100DD000F10421F08AE090E00E940000809110026E
:100DE00081701F928F93A4EAB1E0BF93AF930E94EA
:100DF0004D030F900F900F900F900ACE8630A9F4FC
:100E000090914E03992329F081E09D3419F080E000
:100E100001C0898580930F0241E050E063E071E0FA
:100E20008FE092E00E94B820F3CD833119F40E9444
:100E30004216EECD8231F1F40E940E036D837E8363
:100E40008F83988726E143E06FEF80E00E94BA0B22
:100E5000FC0184818F71806A8483838187708062C2
:100E600083838D819E81AF81B88587839087A18799
:100E7000B287DAC0813001F5A0E0B0E0AB2B09F415
:100E8000C7CD929596959770953049F460914E0331
:100E900070914F0380915003909151030AC09111BA
:100EA00005C08EE493E00E94CA1903C060E070E0C0
:100EB000CB010E940000ACCD8A3009F4A9CD8C3161
:100EC00009F0B4CE80914E03823509F4A1CD863568
:100ED000B1F58EE480937C0066E470E080E090E001
:100EE0000E942F1080917A00806480937A00809114
:100EF0007A0086FDFCCF20907800309079002CE1BC
:100F000043E06FEF80E00E94BA0B8C01FC0184810A
:100F10008F71806684838381877080618383910170
:100F200040E050E0C301B2010E942418D801189695
:100F30003C932E931797C8010E94331669CD8634CF
:100F400009F052C0F8948FEF86BB10928500109282
:100F500084001092800010928200909160002DE039
:100F600088E10FB6F894A895809360000FBE209397
:100F7000600080916000806480936000A89585E0A7
:100F8000809381008091600087FFFCCF10928100E8
:100F9000A8958091600088618093600090936000C4
:100FA000789420908400309085002CE143E06FEF2E
:100FB00080E00E94BA0B8C01FC0184818F718066F5
:100FC00084838381877080618383C101A0E0B0E066
:100FD000BC01CD014BE0660F771F881F991F4A9512
:100FE000D1F7A5019401A0CF8D3401F500917F03C5
:100FF000109180030115110511F403E813E02CE1B1
:1010000043E06FEF80E00E94BA0BFC0184818F7196
:101010008066848383818770806183838B819C81D8
:10102000801B910B90878783CF0186CF853409F091
:10103000EFCC2CE143E06FEF80E00E94BA0B6DE350
:1010400071E00E94A4150E94331600E010E06FEFDB
:10105000C8010E94C8200F5F1F4F0D39B1E01B0768
:10106000B1F780E090E0892B21F08BE090E00E94C6
:10107000000098E088E10FB6F894A895809360008E
:101080000FBE90936000FFCF8A3109F0CFCDC0CC66
:101090002C960FB6F894DEBF0FBECDBFDF91CF9177
:1010A0001F910F91FF90EF90DF90CF90BF90AF9086
:1010B0009F908F907F906F905F904F903F902F9078
:1010C00008950F931F930E940E0320910D02207725
:1010D000203729F000E117E220E030E004C000E60C
:1010E0001AEE20E030E0061717072807390770F4DA
:1010F00082E991E09F938F930E944D030F900F9090
:1011000083E291E01F910F910C9421031F910F91A5
:10111000089580910D02982F9077903759F0982F6D
:1011200092959F709F5F97709295907F8F78892B93
:1011300080930D0280910D02829587701F928F938C
:1011400081E891E09F938F930E944D0380910C0260
:101150008B7F8F7E80930C020F900F900F900F90DB
:1011600080E090E0892B21F087E690E00E9400006B
:1011700083E791E09F938F930E944D030F900F9010
:101180000C941B1680910D028F70863060F08AE5FA
:1011900091E09F938F930E944D030F900F9087E1F2
:1011A00091E00C9421030895809146021F928F9341
:1011B000809145021F928F93809144021F928F93DA
:1011C0008BE391E09F938F930E944D0380910C02DB
:1011D000846080930C0280910D02807880930D02D0
:1011E000E0917D03F0917E038DB79EB708960FB610
:1011F000F8949EBF0FBE8DBF309709F009940895F3
:1012000080910E028F3F79F10E945F146093080273
:101210007093090280930A0290930B028FE291E08F
:101220009F938F930E944D0390910E0280914602EE
:101230000F900F909817A1F01F929F931F928F937A
:1012400087E191E09F938F930E944D0380910E025E
:10125000809346020F900F900F900F900F900F9079
:1012600083E191E025C00E940E03613D7740810536
:10127000910500F180910C02803618F48FE091E026
:1012800017C088E091E09F938F930E944D03809157
:101290000C02877F80930C020F900F9080E090E00B
:1012A000892B21F08AE690E00E94000087E191E01E
:1012B0000C94210308958FEF90E09F938F930E94E9
:1012C0004D030F900F9080E090E0892B21F088E093
:1012D00090E00E9400008FEF80930E0280910C023C
:1012E000886080930C0228E143E06FEF80E00E9469
:1012F000BA0B61E00E9498150C948A038091440215
:101300008F3F99F084EF90E09F938F930E944D035D
:101310000F900F9080E090E0892B21F087E090E023
:101320000E9400008FE091E020C00E940E03613D0A
:10133000774081059105D8F080910C02803618F431
:101340008BE091E012C086EE90E09F938F930E9415
:101350004D030F900F9080E090E0892B21F089E6FB
:1013600090E00E94000087E091E00C942103089532
:101370008EED90E09F938F930E944D030F900F90FE
:10138000809144028F3FE1F480E090E0892B21F0CE
:1013900086E090E00E94000082ED90E09F938F93A2
:1013A0000E944D0323E043E06FEF80E00E94BA0B00
:1013B0006DE471E00E94A4150F900F900C948A03C5
:1013C00008950E940E03613D77408105910520F448
:1013D00080910C0281FF0895809145028F3FC1F0FA
:1013E00085EC90E09F938F930E944D0380910C02B7
:1013F0008E7F80930C020F900F9080E090E0892BFD
:1014000021F085E090E00E9400008BE091E021C097
:1014100080910C02803658F481EA90E09F938F937C
:101420000E944D030F900F9087E191E012C085EB71
:1014300090E09F938F930E944D030F900F9080E058
:1014400090E0892B21F088E690E00E94000087E080
:1014500091E00C94210387E990E09F938F930E9481
:101460004D030F900F9080E090E0892B21F084E0F5
:1014700090E00E94000080910C02897F816080933F
:101480000C028FEF809346028093450227E043E0F1
:101490006FEF0E94BA0B6DE471E00E94A4150C94EA
:1014A0008A03CF93219A229ACFB7F8948091F001C2
:1014B000811127C0E4E9F3E08491E8EAF3E0949134
:1014C000E82FF0E0EE0FFF1FE459FC4FA591B49117
:1014D000EC91E92321F461E08AE00E94C30F61E00E
:1014E0008AE00E94F30F8CB580618CBD8CB580645E
:1014F0008CBD61E08DE00E94F30F61E08BE00E9403
:10150000F30F8091F0018F5F8093F001CFBF299896
:101510002A9A6EE080E20E940A1665E070E080E0A0
:1015200090E00E942F1063E083E20E940A166FE5AC
:1015300084E20E940A166CE485E20E940A1663E2C5
:1015400086E20E940A1663E780E50E940A1666E0BA
:101550008DE30E940A1621E041E060E070E086E041
:101560000E94D915C82F21E041E060E070E085E0DD
:101570000E94D9158C3409F049C0C33209F046C025
:1015800062E082E20E940A1660E081E20E940A168E
:1015900063E08CE30E940A168FEF8093020120E043
:1015A00045E062E071E08BE20E94D91520E045E061
:1015B00062E071E08AE20E94D91520E045E062E035
:1015C00071E080E30E94D91582EE0E942D1681EE13
:1015D0000E942D1660E787E20E940A1686E890E0D6
:1015E0009F938F930E944D0380910C0280618093A2
:1015F0000C02809144020F900F908F3FC1F00E9427
:101600008204811114C087E091E013C082E790E06A
:101610009F938F930E944D030F900F9080E090E076
:10162000892B89F387E690E00E940000ECCF87E1E8
:1016300091E0CF910C94210388E690E09F938F93E3
:101640000E944D03ECE0F2E08081877F8F7E8083F3
:10165000109208021092090210920A0210920B02D4
:101660000F900F9043E050E060E070E084E492E07F
:101670000C94A82020917A002F7720937A00309143
:1016800060008A309105B1F083FD02C028E001C0FE
:1016900028E28770822B98E10FB6F894A895909372
:1016A00060000FBE80936000809160008065809331
:1016B00060000BC00FB6F894A89580916000886117
:1016C00080936000109260000FBE83B7817F8460BA
:1016D00083BFF89483B7816083BF85B7806685BF79
:1016E0008F7D85BF7894889583B78E7F83BFF8946C
:1016F000A8958091600088618093600030936000BD
:10170000789480917A00806880937A0008951F927F
:101710000F920FB60F9211240F900FBE0F901F90D3
:101720001895833081F028F4813099F08230A1F04F
:1017300008958730A9F08830B9F08430D1F48091D1
:1017400080008F7D03C0809180008F778093800020
:10175000089584B58F7702C084B58F7D84BD0895C8
:101760008091B0008F7703C08091B0008F7D80930F
:10177000B0000895E6E2F3E0909144029183828301
:101780006683258347708481807E482B4483CF0104
:1017900008950F931F93CF93DF93EC018C81829573
:1017A0008695877091F44B8146954695469550E015
:1017B000BE01695F7F4F81E192E00E947D19EB815C
:1017C000E695E695E695F0E077C0813031F48F81BB
:1017D0004AE061E172E090E007C0823041F44AE003
:1017E00061E172E08F8198850E94F11968C08330B1
:1017F00041F44AE061E172E08F8198850E944A1AC3
:101800005EC0843051F46F81788589859A852AE09D
:1018100041E152E00E94FC1952C0853051F46F81C1
:10182000788589859A852AE041E152E00E94281A4C
:1018300046C0873071F42B85293008F028E06F818D
:10184000788589859A8501E112E042E00E948C1931
:1018500036C08630A1F520E0EB81E695E695E69569
:101860002E1738F5E22FF0E0AF01440F551FDA01D3
:10187000AF5EBD4FEC0FFD1F8781082E000C990B4A
:1018800034E0959587953A95E1F78F708A3010F49A
:10189000805D01C0895C8C93DA01AE5EBD4F8781AB
:1018A0008F708A3010F4805D01C0895C8C932F5F4B
:1018B000D3CFF0E0EE0FFF1FEF5EFD4F108281E10E
:1018C00092E0DF91CF911F910F91089580914B038A
:1018D000829586958770813019F480914E03089522
:1018E000811105C08EE493E00E94AC19089580E058
:1018F0000895009769F0FC0101900020E9F7319705
:10190000AF01481B590BBC0187E492E00C94B51160
:1019100080E090E008958F929F92AF92BF920F93D4
:101920001F93CF93DF93CDB7DEB7A1970FB6F8948F
:10193000DEBF0FBECDBF19A2423008F44AE08E01CF
:101940000F5D1F4F842E912CA12CB12CA501940169
:101950000E942418E62FB901CA0101501109EA308A
:1019600014F4E05D01C0E95CD801EC93232B242B37
:10197000252B61F7C8010E94790CA1960FB6F89447
:10198000DEBF0FBECDBFDF91CF911F910F91BF90F2
:10199000AF909F908F900895CF93DF93262F8F3F26
:1019A00019F0CDE4D1E002C0C5E4D1E040E0682FF9
:1019B00080E00E94BA0BBE010E94A415DF91CF9176
:1019C0000C943316FC018091440281839481907FB2
:1019D000916094838091100280FF03C0CF010C942A
:1019E000331680E394E09F938F930E944D030F90F2
:1019F0000F9080E00895CF92DF92EF92FF92CF9305
:101A0000DF93D82F0E945F146B017C0181E0D1111C
:101A100080E080934C03C0E00E945F14AB01BC01E6
:101A20004C195D096E097F09403D574061057105FC
:101A300080F4C1110EC0A8950E94C30490914B037D
:101A40009770933049F7C1E080914C038D13E3CF39
:101A5000E3CF8C2FDF91CF91FF90EF90DF90CF906D
:101A600008958F929F92AF92BF92CF92DF92EF92A2
:101A7000FF926B017C011F928FEF8F931F928F93C8
:101A80001F928F931F928F931F921F92FF92EF923C
:101A9000DF92CF9281E094E09F938F930E944D0359
:101AA00080910C022DB73EB7205F3F4F0FB6F894E0
:101AB0003EBF0FBE2DBF82FD34C083EF93E09F93E6
:101AC0008F930E944D030E945F144B015C010F90A5
:101AD0000F9080E090E0DC0120910C0222FD59C0C3
:101AE0008C159D05AE05BF0508F059C0803137E261
:101AF0009307A105B10508F440C0C81AD90AEA0A3B
:101B0000FB0AFF92EF92DF92CF9283EE93E09F93D6
:101B10008F930E944D030F900F900F900F900F9096
:101B20000F9086ED93E09F938F930E944D030E9448
:101B30001B160F900F9080E090E0892B21F08EE033
:101B400090E00E94000087E492E00E948012809161
:101B50001B018F3F31F520E4C2162FE1D206E104CC
:101B6000F104F8F089E090E00E943A0B80E4C81A92
:101B70008FE1D80AE108F108EACFA8950E94C304D2
:101B80000E945F14DC01CB0188199909AA09BB09DD
:101B9000A3CF8C159D05AE05BF0508F4AECF8EEF23
:101BA000D7C080911B018F3F41F430EAC3163FE05C
:101BB000D306E104F10408F072C080911B018F3F4D
:101BC00041F480EDC81687E0D806E104F10408F07E
:101BD00071C080911B018F3F41F428EEC21623E0B3
:101BE000D206E104F10408F070C080911B018F3F20
:101BF00041F434EFC31631E0D306E104F10408F0F8
:101C00006FC080911B018F3F39F48AEFC816D10451
:101C1000E104F10408F06FC080911B018F3F39F49B
:101C20002DE7C216D104E104F10408F06EC08091E2
:101C30001B018F3F39F430E4C316D104E104F104F1
:101C400008F06DC080911B018F3F39F480E2C81607
:101C5000D104E104F10408F06CC080911B018F3FB6
:101C600039F420E1C216D104E104F10408F06BC09C
:101C700080E090E0892B21F08FE090E00E9400004E
:101C80008FEF8F938F9386EC93E09F938F930E94B7
:101C90004D030F900F900F900F908FEF59C088E079
:101CA00090E00E943A0B30EAC31A3FE0D30AE10801
:101CB000F10883CF87E090E00E943A0B80EDC81ACC
:101CC00087E0D80AE108F10884CF86E090E00E941E
:101CD0003A0B28EEC21A23E0D20AE108F10885CFB8
:101CE00085E090E00E943A0B34EFC31A31E0D30A4A
:101CF000E108F10886CF84E090E00E943A0B8AEF79
:101D0000C81AD108E108F10887CF83E090E00E946B
:101D10003A0B28E7C21AD108E108F10888CF82E01F
:101D200090E00E943A0B3CE3C31AD108E108F108A5
:101D300089CF81E090E00E943A0B8EE1C81AD10869
:101D4000E108F1088ACF80E090E00E943A0B90CF42
:101D5000FF90EF90DF90CF90BF90AF909F908F90CB
:101D60000895CF93DF930E94790CEC018BE491E00E
:101D70000E94790C8C0F9D1FDF91CF910895CF9217
:101D8000DF92EF92FF92CF93DF936B017C01E091A2
:101D90004702F09148020190F081E02D6DE287E466
:101DA00092E00995EC0166277727CB016C197D0934
:101DB0008E099F094AE00E948B0C8C0F9D1FDF91BA
:101DC000CF91FF90EF90DF90CF9008954F925F9268
:101DD0006F927F928F929F92AF92BF92CF92DF923B
:101DE000EF92FF926B017C01B42E9B01AC010E942B
:101DF0007319882319F08EE491E027C0260137017A
:101E0000E89477F82FEF3FEF4FE75FE7C301B201A8
:101E10000E94731981110DC02FEF3FEF4FE75FE76D
:101E2000C301B2010E94841F18161CF482E591E0E0
:101E30000CC02FEF3FEF4FE75FE4C701B6010E94F0
:101E40006E19181684F486E591E0FF90EF90DF900C
:101E5000CF90BF90AF909F908F907F906F905F904A
:101E60004F900C94790C2FEF3FEF4FE75FECC701D9
:101E7000B6010E94841F87FDE6CF20E030E0A90173
:101E8000C701B6010E94841F87FF11C0E09147027D
:101E9000F09148020190F081E02D6DE287E492E03C
:101EA00009954C01F7FAF094F7F8F09402C0812CF0
:101EB000912CA12C60E070E080E09FE3AB1441F036
:101EC00020E030E040E251E40E94CD18A394F6CF28
:101ED0009B01AC01C701B6010E9461182B013C01B6
:101EE0000E943F196B017C010E94891F9B01AC017C
:101EF000C301B2010E9460182B013C014AE0C701F6
:101F0000B6010E948B0C7C01E80CF91CBB2031F05F
:101F10008AE591E00E94790CE80EF91EDB2CDD20A9
:101F200021F120E030E040E251E4C301B2010E941F
:101F3000EA1F2B013C010E943F194B01A12CB12C3F
:101F40004AE0C501B4010E948B0CE80EF91EC501E0
:101F5000B4010E94891F9B01AC01C301B2010E9420
:101F600060182B013C01DA94DACFC701FF90EF90A3
:101F7000DF90CF90BF90AF909F908F907F906F90A9
:101F80005F904F9008951F93CF93DF93282F30E0F9
:101F9000F901EE54FC4F8491F901E256FC4FD491C3
:101FA000F901E657FC4FC491CC23C9F0162F8111DB
:101FB0000E94910BEC2FF0E0EE0FFF1FEA58FC4F50
:101FC000A591B4918FB7F894111105C09C91ED2F94
:101FD000E095E92302C0EC91ED2BEC938FBFDF91EC
:101FE000CF911F910895CF93DF9390E0FC01E256CB
:101FF000FC4F2491FC01E657FC4F8491882361F14A
:1020000090E0880F991FFC01E459FC4FC591D491D1
:10201000FC01EA58FC4FA591B491611109C09FB72A
:10202000F8948881209582238883EC912E230BC01D
:10203000623061F49FB7F8943881822F80958323B2
:102040008883EC912E2B2C939FBF06C08FB7F894FA
:10205000E8812E2B28838FBFDF91CF9108958F9237
:102060009F92AF92BF92CF92DF92EF92FF926B015D
:102070007C010E943A144B015C01C114D104E104BB
:10208000F104F1F00E943A14DC01CB01881999099E
:10209000AA09BB09883E9340A105B10570F321E070
:1020A000C21AD108E108F10888EE880E83E0981E74
:1020B000A11CB11CC114D104E104F10419F7DDCF56
:1020C000FF90EF90DF90CF90BF90AF909F908F9058
:1020D00008954F925F927F928F929F92AF92BF929C
:1020E000CF92DF92EF92FF920F931F93CF93DF93E4
:1020F0001F92CDB7DEB7182F0E945F14111124C0B4
:102100000091FE011091FF01209100023091010227
:102110006B017C01C01AD10AE20AF30A2091FA018C
:102120003091FB012130310529F00FEC17E020E060
:1021300030E004C007EE13E020E030E0C016D10626
:10214000E206F30608F4FFC06093FE017093FF01FE
:10215000809300029093010280E090E0A0ECBFE742
:102160008093F1019093F201A093F301B093F401F5
:102170008093F5019093F601A093F701B093F801D5
:1021800060E08091F9010E94C30F61E08091F90144
:102190000E94F30F8091FA019091FB01019739F4AD
:1021A00062E170E080E090E00E942F1004C08CE3B8
:1021B00096E00197F1F760E08091F9010E94F30F3A
:1021C00061E08091F9010E94C30F412C512C00E085
:1021D00010E0C12CD12C3DEF932E0E943A14A62E74
:1021E000892D8170B82EE82E880FFF080E943A14BE
:1021F0006A196B3518F081E090E055C02091F90123
:1022000030E0F901EE54FC4F8491F901E256FC4FA5
:102210008490F901E657FC4F74907720B9F0882339
:1022200021F069830E94910B6981E72DF0E0EE0FA8
:10223000FF1FE058FC4FA591B491EC918E2231E044
:1022400020E009F430E0832F922F02C080E090E07C
:102250008E159F0509F4CACF97FC08C0BB2031F04A
:10226000CC0CDD1C6F3110F06894C0F88FE198162B
:1022700039F08FE3981205C02601C12CD12C01C082
:102280008601939480E59812A8CF612F7727E52CDB
:10229000F12C842D800F860F850D90E08C159D0507
:1022A00039F082E090E09093FD018093FC014BC0F7
:1022B0008091FA019091FB01019791F480E090E008
:1022C0000E94891F6093F5017093F6018093F701D6
:1022D0009093F801B70180E090E00E94891F27C029
:1022E000B80180E090E00E94891F2DEC3CEC4CECA2
:1022F0005DE30E94EA1F6093F5017093F6018093FD
:10230000F7019093F801B20177FF05C07F7744246D
:102310005524461A570AB201550C880B990B0E9496
:102320008B1F2DEC3CEC4CEC5DE30E94EA1F6093AC
:10233000F1017093F2018093F3019093F4011092F4
:10234000FD011092FC010F90DF91CF911F910F9131
:10235000FF90EF90DF90CF90BF90AF909F908F90C5
:102360007F905F904F9008950895CF92DF92EF9203
:10237000FF920F931F93CF93DF936C017A018B0130
:10238000C0E0D0E0CE15DF0589F0D8016D918D0158
:10239000D601ED91FC910190F081E02DC6010995E7
:1023A000892B11F47E0102C02196ECCFC701DF9189
:1023B000CF911F910F91FF90EF90DF90CF900895F4
:1023C000FC01918D828D981761F0828DDF01A80F3D
:1023D000B11D5D968C91928D9F5F9F73928F90E05F
:1023E00008958FEF9FEF0895FC01918D828D9817CE
:1023F00031F0828DE80FF11D858D90E008958FEF0B
:102400009FEF0895FC01918D228D892F90E0805CD3
:102410009F4F821B91098F739927089587E492E05B
:102420000E94021221E0892B09F420E0822F0895F6
:10243000FC01848DDF01A80FB11DA35ABF4F2C9161
:10244000848D90E001968F739927848FA689B78930
:102450002C93A089B1898C9180648C93938D848D09
:10246000981306C00288F389E02D80818F7D8083D8
:102470000895EF92FF920F931F93CF93DF93EC0198
:1024800081E0888F9B8D8C8D981305C0E889F98930
:10249000808185FD24C0F62E0B8D10E00F5F1F4F4D
:1024A0000F731127E02E8C8DE8120CC00FB607FCBD
:1024B000FACFE889F989808185FFF5CFCE010E94A6
:1024C0001812F1CF8B8DFE01E80FF11DE35AFF4F7B
:1024D000F0820B8FEA89FB898081806207C0EE89D8
:1024E000FF896083E889F98980818064808381E045
:1024F00090E0DF91CF911F910F91FF90EF900895A1
:10250000CF93DF93EC01888D8823C9F0EA89FB899A
:10251000808185FD05C0A889B9898C9186FD0FC091
:102520000FB607FCF5CF808185FFF2CFA889B98966
:102530008C9185FFEDCFCE010E941812E7CFDF917D
:10254000CF91089580E090E0892B29F00E940E122F
:1025500081110C94000008950E947819CF92DF92A7
:10256000EF92FF92CF93DF9381E00E94691080E0A9
:102570000E946910C090F101D090F201E090F30147
:10258000F090F401A7019601C701B6010E947319EA
:10259000882329F08CE591E00E94B10E65C020915E
:1025A0007003309171034091720350917303C7011E
:1025B000B6010E94841F811105C080916F038A308B
:1025C00009F04FC0C0927003D0927103E092720381
:1025D000F092730380911D01811110C026E636E64A
:1025E00046EE5FE3C701B6010E94EA1F20E030E03B
:1025F00040E052E40E9461186B017C0110926F036D
:1026000020E030E0A901C701B6010E9461186B010A
:102610007C018091E702877088628093E702809155
:10262000E802806E8093E802C092EB02D092EC0246
:10263000E092ED02F092EE0281E08093EF0284EEF0
:1026400092E00E94E20C81E891E00E94790C42E065
:10265000C701B6010E94E60E8BE491E00E94790C5E
:1026600003C08F5F80936F0380E00E946910C09069
:10267000F501D090F601E090F701F090F801A70184
:102680009601C701B6010E947319882329F085E8D5
:1026900091E00E94B10E47C020916B0330916C0312
:1026A00040916D0350916E03C701B6010E94841FD3
:1026B000811104C080916A038A3091F5C0926B0346
:1026C000D0926C03E0926D03F0926E0310926A0355
:1026D00080910803877088628093080380910903C2
:1026E000806E80930903C0920C03D0920D03E09298
:1026F0000E03F0920F0381E08093100385E093E0D6
:102700000E94E20C86EA91E00E94790C42E0C70147
:10271000B6010E94E60E8BE491E00E94790C03C0A2
:102720008F5F80936A0380911C0120E4829FC00127
:10273000112480937C0080917A00806480937A00D9
:1027400080917A0086FDFCCFC0917800809179005D
:10275000D0E0D82B6E010D2E000CEE08FF08D7FF3D
:1027600005C0C701B6010E94BF0E05C04AE0C701FF
:10277000B6010E948B0C8BE491E00E94790CCE0193
:102780006AE070E00E941018EB018AEA91E00E9472
:10279000790CC701B6010E948B1F29E037E64CE592
:1027A0005BE30E94EA1F42E00E94E60E8CEB91E0A0
:1027B0000E94B10E8FEB91E00E94790CBE010D2EAC
:1027C000000C880B990BD7FF03C00E94BF0E03C0FB
:1027D0004AE00E948B0C81ED91E00E94B10E809145
:1027E0006803909169038C179D0779F020E043E01E
:1027F0006FEF80E00E94BA0B6C2F0E9498150E9428
:102800003316D0936903C093680360E67AEE80E0E4
:1028100090E0DF91CF91FF90EF90DF90CF900C94FC
:10282000310D2BE043E06FEF80E00E94BA0B64EDC6
:1028300071E00E94A4150E9433162CE043E06FEF74
:1028400080E00E94BA0B6BEE71E00E94A4150E941A
:10285000331667E080E00E94CC0C66E081E00E94C5
:10286000CC0C81E090910F02911101C080E0809327
:102870001D0108953FB7F8948091790390917A03F0
:10288000A0917B03B0917C0326B5A89B05C02F3F88
:1028900019F00196A11DB11D3FBFBA2FA92F982F86
:1028A0008827820F911DA11DB11DBC01CD0143E000
:1028B000660F771F881F991F4A95D1F708952FB784
:1028C000F8946091750370917603809177039091ED
:1028D00078032FBF089583E08093F9011092FB01E4
:1028E0001092FA010E945F14DC01CB01885B9B40CF
:1028F000A109B1098093FE019093FF01A09300020A
:10290000B093010282E090E09093FB018093FA0182
:1029100080E00E9469108091FC019091FD0181305E
:10292000910521F49093FB018093FA0183E0809359
:102930001C018091FA019091FB01019719F060ED63
:1029400077E002C068EE73E080E090E00C94310D17
:102950001F920F920FB60F9211242F933F938F93D4
:102960009F93AF93BF938091750390917603A0914D
:102970007703B09178033091740326E0230F2D374D
:1029800020F40296A11DB11D05C029E8230F03966E
:10299000A11DB11D2093740380937503909376035A
:1029A000A0937703B09378038091790390917A0391
:1029B000A0917B03B0917C030196A11DB11D809372
:1029C000790390937A03A0937B03B0937C03BF9128
:1029D000AF919F918F913F912F910F900FBE0F90CC
:1029E0001F9018951F920F920FB60F9211242F93DC
:1029F0003F934F935F936F937F938F939F93AF9387
:102A0000BF93EF93FF93E0912001F091210109958D
:102A1000FF91EF91BF91AF919F918F917F916F91B6
:102A20005F914F913F912F910F900FBE0F901F908C
:102A300018951F920F920FB60F9211242F933F9368
:102A40004F935F936F937F938F939F93AF93BF93B6
:102A5000EF93FF93E0911E01F0911F010995FF9103
:102A6000EF91BF91AF919F918F917F916F915F9106
:102A70004F913F912F910F900FBE0F901F9018957F
:102A80001F920F920FB60F9211242F933F934F93E3
:102A90005F936F937F938F939F93AF93BF93EF93C6
:102AA000FF9387E492E00E941812FF91EF91BF918B
:102AB000AF919F918F917F916F915F914F913F91D6
:102AC0002F910F900FBE0F901F9018951F920F928D
:102AD0000FB60F9211242F938F939F93EF93FF9331
:102AE000E0915702F09158028081E0915D02F091EF
:102AF0005E0282FD12C09081809160028F5F8F73B1
:102B000020916102821751F0E0916002F0E0E95BF0
:102B1000FD4F958F8093600201C08081FF91EF91FE
:102B20009F918F912F910F900FBE0F901F9018952E
:102B3000FC01838187708860838384818F718062C8
:102B400084836783CF0108950F931F93CF93DF93FF
:102B5000EC016115710561F0FB0101900020E9F7BE
:102B60003197E61BF70BE931F10518F0E9E101C0F7
:102B7000E0E00E2F10E0C80123E0880F991F2A958E
:102B8000E1F79B819770892B8B838C818F718C836C
:102B9000EE2329F0A801CE0107960E947D19FE01BF
:102BA000E00FF11F1782CE01DF91CF911F910F919E
:102BB000089590E59CBD1DBC2A98E0E1F0E03197B6
:102BC000F1F78EBD00000DB407FEFDCF8EB5FB0101
:102BD0009FEF4150C8F0222361F09EBD00000DB46C
:102BE00007FEFDCF8EB56115710599F3808331968F
:102BF000F0CFDF01119680818EBD00000DB407FE7D
:102C0000FDCF8EB5FD01E5CF2A9AE0E1F0E03197E6
:102C1000F1F70895CF93DF931F92CDB7DEB76983A5
:102C200020E041E0BE016F5F7F4F0E94D9150F90F9
:102C3000DF91CF91089529986CE080E20C940A16F8
:102C40006FE080E20E940A16609122016F3F19F046
:102C50008AE20E940A16299A089520E040E060E086
:102C600070E00C94D91520910C0222FD0C948A037B
:102C700087E494E09F938F930E944D030F900F90F1
:102C800080E00895CF9380E090E0892B21F08CE0E4
:102C900090E00E9400002FE043E06FEF80E00E9490
:102CA000BA0B6DE471E00E94A4158091290387702E
:102CB00080618093290380912A038F71806C8093B7
:102CC0002A0381E080932D0310922E0386E293E085
:102CD0000E9433168FE00E94FB0C61E18FEF0E948F
:102CE000CC0CC091450226E043E06FEF80E00E94EB
:102CF000BA0B6C2F0E9498150E94331686E00E9432
:102D0000FB0CCF910C941114CF938091100281FD94
:102D10002FC00E94421685E594E09F938F930E94F6
:102D20004D030F900F9080E090E0892B21F089E017
:102D300090E00E9400008091100281608093100258
:102D4000C4E02AE143E06FEF80E00E94BA0B62E04A
:102D50000E9498150E9433168BE10E94FB0C811192
:102D600002C0C15071F780911002826080931002FE
:102D7000CF910895CF93E7E4F2E01382128288EEB8
:102D800093E0A0E0B0E084839583A683B78381E3DA
:102D900091E09183808385EC90E09587848784EC33
:102DA00090E09787868780EC90E0918B808B81EC18
:102DB00090E0938B828B82EC90E0958B848B86ECF9
:102DC00090E0978B868B118E128E138E148E87E473
:102DD00093E00E94FB1786E293E00E94FB1785E0D8
:102DE00093E00E94FB17E5E0F3E01682C1E0C583A3
:102DF00084EE92E00E94FB17E4EEF2E0C6831582B7
:102E0000CF910895789484B5826084BD84B5816043
:102E100084BD85B5826085BD85B5816085BD8091A5
:102E20006E00816080936E0010928100809181001D
:102E30008260809381008091810081608093810015
:102E4000809180008160809380008091B1008460D7
:102E50008093B1008091B00081608093B000809138
:102E60007A00846080937A0080917A0082608093F7
:102E70007A0080917A008E7F80937A0080917A0028
:102E8000806880937A001092C100A89580E090E05D
:102E9000892B11F00E940000E0915702F091580236
:102EA00082E08083E0915302F09154021082E0911D
:102EB0005502F091560288E0808310925F02E09103
:102EC0005B02F0915C0286E08083E0915902F09110
:102ED0005A02808180618083E0915902F0915A0208
:102EE000808188608083E0915902F0915A0280814C
:102EF00080688083E0915902F0915A0280818F7D31
:102F0000808384EA94E09F938F930E944D03809185
:102F100010028D7F809310020F900F9080E090E060
:102F2000892B51F087E994E09F938F930E944D0382
:102F30000E9400000F900F9041E050E063E071E0CC
:102F40008FE092E00E94A8206FEF81E090E00E9465
:102F5000C82080910D028F7880930D021092030299
:102F60001092020283E291E00E94210384E896E13C
:102F700090937E0380937D031F921F921F921F9256
:102F800082E694E09F938F930E944D030E945F140A
:102F90000F900F900F900F900F900F900E945F1462
:102FA0000E94C304A89580910C0282FFF7CF8AE8A3
:102FB00094E09F938F930E944D030E946B140F9097
:102FC0000F9080910C0282FB882780F91F928F93CB
:102FD00082E794E09F938F930E944D03A8950F90F2
:102FE0000F900F900F90A8950E94C3040E94AE12FC
:102FF0000E94A212F8CFCF93DF93FC0110821182BE
:103000001282148215821682DC0117968AE1ED0184
:1030100019928A95E9F782E08383DF91CF91089531
:1030200097FB072E16F4009407D077FD09D00E9475
:10303000461807FC05D03EF4909581959F4F089562
:10304000709561957F4F0895A1E21A2EAA1BBB1BB4
:10305000FD010DC0AA1FBB1FEE1FFF1FA217B30764
:10306000E407F50720F0A21BB30BE40BF50B661F7A
:10307000771F881F991F1A9469F76095709580953E
:1030800090959B01AC01BD01CF010895AA1BBB1B0C
:1030900051E107C0AA1FBB1FA617B70710F0A61B58
:1030A000B70B881F991F5A95A9F780959095BC0179
:1030B000CD010895EE0FFF1F0590F491E02D0994C6
:1030C0005058BB27AA270E9478180C946E200E94A3
:1030D000602038F00E94672020F039F49F3F19F4F7
:1030E00026F40C945D200EF4E095E7FB0C94572039
:1030F000E92F0E947F2058F3BA17620773078407ED
:10310000950720F079F4A6F50C94A1200EF4E09533
:103110000B2EBA2FA02D0B01B90190010C01CA0191
:10312000A0011124FF27591B99F0593F50F4503E3C
:1031300068F11A16F040A22F232F342F4427585F2E
:10314000F3CF469537952795A795F0405395C9F746
:103150007EF41F16BA0B620B730B840BBAF09150FE
:10316000A1F0FF0FBB1F661F771F881FC2F70EC09D
:10317000BA0F621F731F841F48F487957795679570
:10318000B795F7959E3F08F0B0CF9395880F08F05C
:103190009927EE0F9795879508950E94E1180C9452
:1031A0006E200E94672058F00E94602040F029F4B1
:1031B0005F3F29F00C94572051110C94A2200C94DD
:1031C0005D200E947F2068F39923B1F3552391F38A
:1031D000951B550BBB27AA2762177307840738F086
:1031E0009F5F5F4F220F331F441FAA1FA9F335D0E3
:1031F0000E2E3AF0E0E832D091505040E695001C97
:10320000CAF72BD0FE2F29D0660F771F881FBB1F50
:10321000261737074807AB07B0E809F0BB0B802D2E
:10322000BF01FF2793585F4F3AF09E3F510578F05A
:103230000C9457200C94A2205F3FE4F3983ED4F303
:10324000869577956795B795F7959F5FC9F7880F2E
:10325000911D9695879597F90895E1E0660F771F80
:10326000881FBB1F621773078407BA0720F0621B11
:10327000730B840BBA0BEE1F88F7E09508950E943C
:10328000872088F09F5798F0B92F9927B751B0F051
:10329000E1F0660F771F881F991F1AF0BA95C9F7DA
:1032A00014C0B13091F00E94A120B1E008950C94B7
:1032B000A120672F782F8827B85F39F0B93FCCF36A
:1032C000869577956795B395D9F73EF49095809557
:1032D000709561957F4F8F4F9F4F08950E94C61F35
:1032E00008F48FEF08950E94C61F880B990B08956C
:1032F00081E090E0F8940C941121FB01DC01415035
:10330000504048F001900D920020C9F701C01D9275
:1033100041505040E0F70895EF920F931F93CF93E1
:10332000DF93E80147FD02C034E001C034E1E42F3F
:10333000440FFF0BF7FF03C0F195E195F109E32E70
:10334000022F2E2FAE010E94621CCE01DF91CF9181
:103350001F910F91EF900895FC0188279927E89419
:1033600021912032E9F3293010F02E30C8F32B32AE
:1033700041F02D3239F4689404C00E94201A820F63
:10338000911D219120532A30C0F31EF49095819510
:103390009F4F08951F93FC0199278827BC01E8944B
:1033A00011911032E9F3193010F01E30C8F31B32BE
:1033B00051F01D3249F4689406C00E940B1A610F47
:1033C000711D811D911D119110531A30B0F33EF4FF
:1033D00090958095709561957F4F8F4F9F4F1F916E
:1033E0000895BB274A3031F4992322F4BDE2909529
:1033F00081959F4F0C944B1ABB272A3051F4992387
:1034000042F4BDE290958095709561957F4F8F4F06
:103410009F4F0C94291A592F482F372F262F660FAC
:10342000771F881F991F660F771F881F991F620FCC
:10343000731F841F951F660F771F881F991F08959C
:103440007AE0979F902D879F802D910D11240895EC
:10345000BB27FA01A62F6217710581059105330B71
:1034600030FB66F0AA27660F771F881F991FAA1FD7
:10347000A21710F0A21B63953850A9F7A05DAA33DC
:1034800008F0A95DA19336F7B111B1931082CA017A
:103490000C94DE1EBB27FB015527AA27880F991F16
:1034A000AA1FA41710F0A41B83955051B9F7A05D73
:1034B000AA3308F0A95DA193009779F7B111B193F0
:1034C0001192CB010C94DE1EAEE0B0E0EAE6FAE128
:1034D0000C94E8208C01CA014EE04C831A830983C6
:1034E00077FF02C060E070E8FB013197FE83ED8357
:1034F000A901BC01CE0101960E94901A4D815E8106
:1035000057FD0AC02F813885421753070CF49A01E2
:10351000F801E20FF31F10822E96E4E00C940421D0
:10352000ACE0B0E0E6E9FAE10C94DA207C016B0152
:103530008A01FC0117821682838181FFBDC1CE0101
:1035400001964C01F7019381F60193FD859193FF5C
:1035500081916F01882309F4ABC1853239F493FD61
:10356000859193FF81916F01853229F4B70190E035
:103570000E94EE1EE7CF512C312C20E02032A0F427
:103580008B3269F030F4803259F0833269F4206173
:103590002CC08D3239F0803339F4216026C022608E
:1035A000246023C0286021C027FD27C030ED380FDC
:1035B0003A3078F426FF06C0FAE05F9E300D112401
:1035C000532E13C08AE0389E300D1124332E206212
:1035D0000CC08E3221F426FD6BC1206406C08C36EF
:1035E00011F4206802C0883641F4F60193FD8591FC
:1035F00093FF81916F018111C1CF982F9F7D9554C9
:10360000933028F40C5F1F4FFFE3F9830DC083361E
:1036100031F0833771F0833509F05BC022C0F801C7
:10362000808189830E5F1F4F44244394512C5401A1
:1036300015C03801F2E06F0E711CF801A080B18056
:1036400026FF03C0652D70E002C06FEF7FEFC5015C
:103650002C870E94D31E2C0183012C852F77222ECC
:1036600017C03801F2E06F0E711CF801A080B18024
:1036700026FF03C0652D70E002C06FEF7FEFC5012C
:103680002C870E94C81E2C012C852068222E8301C5
:1036900023FC1BC0832D90E048165906B0F4B701F7
:1036A00080E290E00E94EE1E3A94F4CFF50127FCF0
:1036B000859127FE81915F01B70190E00E94EE1E87
:1036C00031103A94F1E04F1A51084114510471F746
:1036D000E5C0843611F0893639F5F80127FF07C0B7
:1036E00060817181828193810C5F1F4F08C060816E
:1036F0007181072E000C880B990B0E5F1F4F2F76E0
:10370000722E97FF09C090958095709561957F4FB7
:103710008F4F9F4F2068722E2AE030E0A4010E9454
:10372000261FA82EA81844C0853729F42F7EB22E54
:103730002AE030E025C0F22FF97FBF2E8F36C1F08E
:1037400018F4883579F0B4C0803719F0883721F043
:10375000AFC02F2F2061B22EB4FE0DC08B2D846020
:10376000B82E09C024FF0AC09F2F9660B92E06C04C
:1037700028E030E005C020E130E002C020E132E086
:10378000F801B7FE07C060817181828193810C5F6F
:103790001F4F06C06081718180E090E00E5F1F4F77
:1037A000A4010E94261FA82EA818FB2DFF777F2EAC
:1037B00076FE0BC0372D3E7FA51450F474FE0AC070
:1037C00072FC08C0372D3E7E05C0BA2C372D03C0D1
:1037D000BA2C01C0B52C34FF0DC0FE01EA0DF11D5D
:1037E0008081803311F4397E09C032FF06C0B39462
:1037F000B39404C0832F867809F0B39433FD13C0CB
:1038000030FF06C05A2CB31418F4530C5B18B32CB9
:10381000B31468F4B70180E290E03C870E94EE1E8A
:10382000B3943C85F5CFB31410F43B1801C0312C90
:1038300034FF12C0B70180E390E03C870E94EE1E87
:103840003C8532FF17C031FD03C088E790E002C01D
:1038500088E590E0B7010CC0832F867859F031FFDE
:1038600002C08BE201C080E237FD8DE2B70190E03B
:103870000E94EE1EA51438F4B70180E390E00E9488
:10388000EE1E5A94F7CFAA94F401EA0DF11D80813F
:10389000B70190E00E94EE1EA110F5CF332009F48D
:1038A00051CEB70180E290E00E94EE1E3A94F6CF2E
:1038B000F7018681978102C08FEF9FEF2C96E2E19E
:1038C0000C94F6204F925F926F927F929F92AF92EC
:1038D000BF92CF92DF92EF92FF920F931F93CF93FD
:1038E000DF93CDB7DEB729970FB6F894DEBF0FBED2
:1038F000CDBF6A01122FB02E2BE3201720F0FF243A
:10390000F394F00E02C0BCE3FB2E0F2D27E0AE01B6
:103910004F5F5F4F0E94F01DAC018981982F997015
:10392000913031F0E1FC06C0E0FE06C090E205C037
:103930009DE203C09BE201C090E0EE2DE07183FFA9
:103940003CC0911102C083E001C084E0811718F4EB
:10395000212F281B01C020E0E1110BC0F601822FAE
:1039600030E2882319F031938150FBCFC20ED11C75
:1039700020E0992329F0D6019C93F60131966F013E
:10398000C6010396E2FE0AC03EE4D6013C9341E440
:1039900011964C93119712963C9306C03EE6F601A1
:1039A000308341E641833283FC01322F40E23323EE
:1039B00009F442C041933150FACF82FF44C09111C3
:1039C00002C083E001C084E0811718F4212F281B76
:1039D00001C020E0E1110BC0F601822F30E2882304
:1039E00019F031938150FBCFC20ED11C20E09923F6
:1039F00029F0D6019C93F60131966F01C60103961A
:103A0000E2FE0BC039E4D6013C933EE411963C93B0
:103A1000119736E412963C9307C039E6F6013083DD
:103A20003EE6318336E63283FC01322F40E2332317
:103A300019F041933150FBCFFC01E20FF11D1082D0
:103A40008EEF9FEFB7C0F1E0911101C0F0E06F2F52
:103A500070E01416150624F49A012F5F3F4F02C040
:103A600021E030E0260F371FBB2029F06B2D70E0DE
:103A70006F5F7F4F02C060E070E0260F371F612F3D
:103A800070E0261737071CF4121B212F01C020E01D
:103A90003E2D387159F4D601322F60E2332319F0EC
:103AA0006D933150FBCFC20ED11C20E0FF2331F0CB
:103AB000D6019C93B6016F5F7F4F6B01E1110BC084
:103AC000F601922F30E3992319F031939150FBCFF7
:103AD000C20ED11C20E09F2D940F3A81782F707177
:103AE000A72E84FF03C0313309F49150191624F432
:103AF000993018F098E001C091E0E42F852F57FF2E
:103B000002C0E0E080E06E2F782FE0E0F0E0AEE26F
:103B10009A2E3A01691A71082A01461A570A0B2D82
:103B200010E01195019511096F3F8FEF780729F487
:103B3000D6019C92C60101966C014617570784F086
:103B4000661677066CF47F01E40CF51CA1E0B0E08A
:103B5000AC0FBD1FEA0EFB1ED7011196BC9002C030
:103B600090E3B92E615071093196C60101967C012E
:103B70006017710724F0D601BC926C01D5CF641791
:103B8000750741F4363320F4353321F4A11002C017
:103B900081E3B82EF601B082F701822F90E28823EC
:103BA00019F091938150FBCFF701E20FF11D1082C4
:103BB00080E090E029960FB6F894DEBF0FBECDBF2F
:103BC000DF91CF911F910F91FF90EF90DF90CF90F9
:103BD000BF90AF909F907F906F905F904F900895AF
:103BE000283008F027E03327DA01990F311D87FDCF
:103BF000916000966105710539F432602E5F3D9346
:103C000030E32A95E1F708959F3F30F08038710541
:103C1000610509F03C5F3C5F3D93913008F080689E
:103C2000911DDF93CF931F930F93FF92EF92192F64
:103C3000987F9695E92F96959695E90FFF27EA5D6F
:103C4000FA4F99273327EE24FF24A701E7010590B7
:103C50000894079428F4360FE71EF81E491F511DDB
:103C6000660F771F881F991F0694A1F70590079488
:103C700028F4E70EF81E491F561FC11D770F881F35
:103C8000991F661F0694A1F70590079428F4F80E73
:103C9000491F561FC71FD11D880F991F661F771F09
:103CA0000694A1F70590079420F4490F561FC71FEB
:103CB000D81F990F661F771F881F0694A9F7849154
:103CC0001095177041F0D695C79557954795F7947D
:103CD000E7941A95C1F7ECECF4E06894159015910F
:103CE00035916591959105907FE27395E118F10A00
:103CF000430B560BC90BD009C0F7E10CF11E431F53
:103D0000561FC91FD01D7EF4703311F48A95E6CF7B
:103D1000E894015030F0080F0AF40027021708F465
:103D2000202F2395022F7A3328F079E37D932A956B
:103D3000E9F710C07D932A9589F6069497956795C3
:103D4000379517951794E118F10A430B560BC90BD9
:103D5000D00998F023957E9173957A3308F070E33B
:103D60007C932013B8F77E9170617D9330F083953A
:103D700071E37D9370E32A95E1F71124EF90FF90B2
:103D80000F911F91CF91DF91992787FD909508950D
:103D9000FC010590615070400110D8F78095909516
:103DA0008E0F9F1F0895FC0161507040019001101B
:103DB000D8F7809590958E0F9F1F0895DC01FC0128
:103DC000672F71917723E1F7329704C07C916D934F
:103DD00070836291AE17BF07C8F308950F931F93C6
:103DE000CF93DF93FB01238121FD03C08FEF9FEF72
:103DF00028C022FF16C04681578124813581421791
:103E0000530744F4A081B1819D012F5F3F4F31835F
:103E100020838C93268137812F5F3F4F3783268302
:103E200010C0EB01092F182F0084F185E02D0995B2
:103E3000892BE1F68E819F8101969F838E83812F4E
:103E4000902FDF91CF911F910F910895FA01AA272A
:103E5000283051F1203181F1E8946F936E7F6E5FCD
:103E60007F4F8F4F9F4FAF4FB1E03ED0B4E03CD07B
:103E7000670F781F891F9A1FA11D680F791F8A1F5E
:103E8000911DA11D6A0F711D811D911DA11D20D0C5
:103E900009F468943F912AE0269F11243019305D7F
:103EA0003193DEF6CF010895462F4770405D419370
:103EB000B3E00FD0C9F7F6CF462F4F70405D4A33BD
:103EC00018F0495D31FD4052419302D0A9F7EACF85
:103ED000B4E0A6959795879577956795BA95C9F7B4
:103EE00000976105710508959B01AC010A2E0694A7
:103EF0005795479537952795BA95C9F7620F731F60
:103F0000841F951FA01D08950E94C61F08F481E01C
:103F10000895E89409C097FB3EF4909580957095BC
:103F200061957F4F8F4F9F4F9923A9F0F92F96E905
:103F3000BB279395F695879577956795B795F1117A
:103F4000F8CFFAF4BB0F11F460FF1BC06F5F7F4F17
:103F50008F4F9F4F16C0882311F096E911C0772329
:103F600021F09EE8872F762F05C0662371F096E832
:103F7000862F70E060E02AF09A95660F771F881F01
:103F8000DAF7880F9695879597F90895990F0008A5
:103F9000550FAA0BE0E8FEEF16161706E807F9071B
:103FA000C0F012161306E407F50798F0621B730BB6
:103FB000840B950B39F40A2661F0232B242B252B37
:103FC00021F408950A2609F4A140A6958FEF811DDA
:103FD000811D08950E94FD1F0C946E200E94602098
:103FE00038F00E94672020F0952311F00C945720A0
:103FF0000C945D2011240C94A2200E947F2070F369
:10400000959FC1F3950F50E0551F629FF001729F7D
:10401000BB27F00DB11D639FAA27F00DB11DAA1F8C
:10402000649F6627B00DA11D661F829F2227B00DD9
:10403000A11D621F739FB00DA11D621F839FA00D64
:10404000611D221F749F3327A00D611D231F849FB4
:10405000600D211D822F762F6A2F11249F5750400B
:104060009AF0F1F088234AF0EE0FFF1FBB1F661F86
:10407000771F881F91505040A9F79E3F510580F04F
:104080000C9457200C94A2205F3FE4F3983ED4F3A5
:10409000869577956795B795F795E7959F5FC1F7F3
:1040A000FE2B880F911D9695879597F9089597F99E
:1040B0009F6780E870E060E008959FEF80EC0895CE
:1040C00000240A94161617061806090608950024F7
:1040D0000A9412161306140605060895092E039471
:1040E000000C11F4882352F0BB0F40F4BF2B11F4E5
:1040F00060FF04C06F5F7F4F8F4F9F4F089557FD44
:104100009058440F551F59F05F3F71F04795880F45
:1041100097FB991F61F09F3F79F0879508951216DC
:1041200013061406551FF2CF4695F1DF08C0161688
:1041300017061806991FF1CF869571056105089439
:104140000895E894BB2766277727CB0197F9089550
:10415000DC01CB01FC01F999FECF06C0F2BDE1BD47
:10416000F89A319600B40D9241505040B8F7089536
:10417000DC01A40FB51F4150504048F0CB01840F23
:10418000951F2E910E94C92041505040D0F70895AC
:10419000262FF999FECF92BD81BDF89A019700B400
:1041A000021639F01FBA20BD0FB6F894FA9AF99AA0
:1041B0000FBE08952F923F924F925F926F927F921F
:1041C0008F929F92AF92BF92CF92DF92EF92FF9227
:1041D0000F931F93CF93DF93CDB7DEB7CA1BDB0BD3
:1041E0000FB6F894DEBF0FBECDBF09942A88398878
:1041F00048885F846E847D848C849B84AA84B9847F
:10420000C884DF80EE80FD800C811B81AA81B9818A
:10421000CE0FD11D0FB6F894DEBF0FBECDBFED019E
:064220000895F894FFCFA1
:10422600FFFF00FCE1A8A889086108B8097E095BC0
:10423600090009D408C2082B0AE109FF0101B411DB
:10424600B411FF1C0B510A0000830380000000001C
:10425600003912B5110212E011F41180124F4B0011
:104266004E41434B00322E312E30000D0A006E6156
:104276006E00696E66006F7666002E004661696C98
:1042860065642072656164696E672074656D70652A
:104296007261747572652066726F6D204448542190
:1042A60000543A20004661696C6564207265616459
:1042B600696E672068756D69646974792066726FC6
:1042C6006D2044485400483A200042617474657277
:1042D6007920566F6C746167653A2000205600425B
:1042E6006174746572792070657263656E743A20C4
:1042F6000020250054656D706572617475726541A4
:104306006E6448756D696469747900312E310000F8
:00000001FF
